:10000000D228A4008417800484138E010C1C8E0057
:1000100023200319CD2823200319CD282320CD2800
:10002000A40059200C080D040319CD28C7208413FF
:100030002408800664001C281D288C0A03198D0FD3
:100040001A288006CD2824088E0601308C008D01E8
:10005000000824050E06031D08008C0A03198D0FE5
:10006000282808008F002608840024095A208413B9
:100070008F080319CD28F03091000E0880389000C9
:10008000F03091030319910003198F030319CD2850
:1000900049285D2003010C1824088E1F24088E08AF
:1000A00003190301900F562880063D2857280000A9
:1000B0004028FF3A84178005CD280D080C04031949
:1000C0008C0A80300C1A8D060C198D068C188D0642
:1000D0000D0D8C0D8D0DCD288F018E00FF308E07FC
:1000E000031C8F07031CCD2803308D00DF307A20DE
:1000F0006E288D01E83E8C008D09FC30031C83289E
:100100008C07031880288C0764008D0F80280C183A
:1001100089288C1C8D2800008D2808008E00033053
:1001200094288E000630942894000F080D02031DB9
:100130009B280E080C02043003180130031902300A
:100140001405031DFF30CD280038031DFF300405C2
:10015000031DFF30CD2891019001103092000D0D4C
:10016000900D910D0E0890020F08031C0F0F9102C5
:100170000318C1280E0890070F0803180F0F9107E6
:1001800003108C0D8D0D920BAF280C08CD288C0917
:100190008D098C0A03198D0A080083130313831237
:1001A000640008008316850108308600831206115A
:1001B000831606118312061083160610831286100A
:1001C000831686108312812128088C0029088D004F
:1001D0008F010F308E209E0028088C0029088D008A
:1001E0008F0114309120A0001E0884002008A42054
:1001F000A000A100640020082104031908290610AA
:100200008316061083128610831686108312E32845
:1002100028088C0029088D008F0114309120031DBF
:100220001A29061483160610831286108316861068
:1002300083122F2128088C0029088D008F010F3090
:100240008E20031D2C290610831606108312861497
:100250008316861083125821E32863002D29063067
:10026000A6001030A4005A308E00013032205030E9
:100270008E00023032207D308E00013032205A3024
:100280008E000230322064308E0002303220AA30DC
:10029000AF00AB21A030AE00A030B000AB21643085
:1002A000AF00AB217830AE007830B000AB21080051
:1002B0000630A6001030A4005A308E0001303220E3
:1002C00050308E00023032207D308E0001303220DE
:1002D0005A308E000230322064308E0002303220DC
:1002E000AA30AF00AB217830AE007830B000AB213F
:1002F0006430AF00AB21A030AE00A030B000AB2125
:10030000080001308C008D0106308400043010207C
:1003100001308C0006308400083001200C08AC004D
:100320000D08AD002C088C002D088D000F308E00BC
:100330008F01AB20AA000D08AB002C088C002D0803
:100340008D0006308E008F01AB20A8000D08A9009B
:1003500001306C2008000130B10064000B30310224
:100360000318CB292F088C008D01063084008030C3
:1003700010202E088C008D010630840040301020A3
:1003800030088C008D0106308400203010200D30A4
:080390006C20B10FAD2908003B
:02400E00F53F7C
:00000001FF
